:100000000C9417060C942C290C9459290C943F0637
:100010000C943F060C943F060C943F060C943F064C
:100020000C943F060C943F060C94C00C0C943F06B5
:100030000C943F060C943F060C943F060C943F062C
:100040000C9486290C943F060C94402D0C947B2D27
:100050000C943F060C943F060C943F060C943F060C
:100060000C943F060C943F06931C9A1C9A1C931CFC
:100070009A1C9A1C9A1C9A1C9A1C9A1C9A1C9A1CD0
:100080009A1C9A1C9A1C9A1C9A1C081C9A1C9A1C52
:100090009A1C9A1C9A1C6B1B9A1C9A1C9A1C9A1CE0
:1000A0009A1C9A1C9A1C9A1C9A1C9A1C9A1C9A1CA0
:1000B0009A1C9A1C9A1C141C141C141C141C141C2E
:1000C000141C141C141C141C9A1C9A1C9A1C9A1C98
:1000D0009A1C9A1C701B131C131C131C131C9A1CB7
:1000E000241C2C1C341C3C1C441C4C1C541C5C1C30
:1000F000661C701C7A1C841CB71B771B9A1C9A1CEC
:100100009A1C9A1C081C9A1C9A1C9A1C9A1C9A1CD1
:100110009A1C9A1C9A1C121C121C121C121C9A1C4F
:10012000241C2C1C341C3C1C441C4C1C541C5C1CEF
:10013000661C701C7A1C841CB71B771B9A1C9A1CAB
:100140009A1C9A1C081CCB1CCB1CCB1CCB1CCB1C9C
:10015000CB1CCB1CCB1CCB1CCB1CCB1CCB1CCB1C67
:10016000EB1DEB1DEB1DEB1DEB1DEB1D121D1C1DF7
:10017000261D301D961DA01DAE1DBF1D5C1ECC1E74
:100180009D1EA21EA71EAC1EB11EB61EBB1ECC1EFF
:10019000C61ED025E525F125FA2507262D2635266C
:1001A00058264526456E746572206D656E752E2E37
:1001B0002E00546F67676C6564206D6963726F50C1
:1001C000504D00546F67676C656420696E76657288
:1001D0007465642050504D2100546F67676C6564EE
:1001E000205458206D7574696E672100546F6767DD
:1001F0006C65642074656C656D657472792100505E
:10020000726F746F636F6C206572726F72207769A2
:1002100074682052580054696D656F757420776852
:10022000656E20636F6E6E656374696E6720746FB0
:1002300020525800507265737320616E79206B658F
:100240007920746F2063616E63656C00436F6E6E1E
:10025000656374696E6720746F2052582C20706F2C
:100260007765722075702074686520525820287751
:100270006974682062696E6420706C7567206966B5
:10028000206E6F74207573696E6720616C77617979
:10029000732062696E642900546F67676C6564201F
:1002A00027696D6D656469617465206F757470751B
:1002B000742700546F67676C65642027736C6176E0
:1002C00065206D6F64652700546F67676C656420F7
:1002D00027616C776179732062696E642700546FBF
:1002E00067676C65642050504D206368616E6E6571
:1002F0006C206C696D6974005365742052535349C6
:1003000020696E6A656374696F6E206368616E6EE2
:10031000656C2028303D3D64697361626C6529001D
:100320005365742050504D206D696E696D756D2058
:1003300073796E630053657420626561636F6E202C
:10034000696E74657276616C0053657420626561D4
:10035000636F6E2064656C6179005365742062651B
:1003600061636F6E206672657175656E6379206971
:100370006E20487A3A20303D64697361626C652C66
:100380002050783D504D52206368616E6E656C2040
:10039000782C2046783D465253206368616E6E6526
:1003A0006C2078005365742050574D2073746F7023
:1003B0002064656C61792028302064697361626C07
:1003C00065642C20312D323535203D3D20302E31D5
:1003D00073202D2035306D696E29005365742050CF
:1003E000504D2073746F702064656C6179202830E3
:1003F0002064697361626C65642C20312D3235355F
:10040000203D3D20302E3173202D2035306D696E1A
:100410002900536574206661696C736166652064A8
:10042000656C61792028302064697361626C656451
:100430002C20312D323535203D3D20302E3173209A
:100440002D2035306D696E29002A2A2A2A2A2A2A67
:100450002A2A2A2A2A2A2A2A2A2A2A2A2A2A2A2AFC
:100460002A2A2A2A2A2A0052582041636B656420CE
:100470002D2072657665727420737563636573737E
:1004800066756C21002A2A2A2A2A2A2A2A2A2A2A36
:100490002A2A2A2A2A2A2A2A2A2A2A2A2A2A2A2ABC
:1004A0002A2A002A2A2A2A2A2A2A2A2A2A2A2A2AD6
:1004B0002A2A2A2A2A2A2A2A2A2A2A2A2A2A2A2A9C
:1004C0000052582041636B6564202D207570646173
:1004D0007465207375636365737366756C21002A98
:1004E0002A2A2A2A2A2A2A2A2A2A2A2A2A2A2A2A6C
:1004F0002A2A2A2A2A2A2A2A2A2A2A2A0056616CE1
:1005000069642063686F69636573206172653A206E
:100510005B315D2D5B31365D20286368616E6E65F1
:100520006C20312D31362900536574206F7574703D
:10053000757420666F7220706F727420005B585D56
:100540002061626F7274206368616E6765732061F9
:100550006E64206578697420525820636F6E6669F6
:1005600067005B535D207361766520736574746901
:100570006E677320746F205258005B525D20726565
:10058000766572742052582073657474696E67734F
:1005900020746F2064656661756C747300557365B3
:1005A000206E756D62657273205B312D445D207421
:1005B0006F206564697420706F727473205B452DC1
:1005C000515D20666F722073657474696E67730085
:1005D000202D20726563656976657220636F6E6693
:1005E0006967757261746F722C207278207377203E
:1005F000000A0A6F70656E4C52536E672000536597
:10060000742073657269616C2062617564726174D3
:10061000653A200056616C69642063686F696365A0
:10062000733A2031202D20342B34202F2032202DDE
:100630002038202F2033202D20382B34202F203419
:10064000202D203132202F2035202D2031322B3407
:10065000202F2036202D203136005365742043682A
:10066000616E6E656C20636F6E6669673A20005339
:1006700065742044617461726174652028302D3284
:10068000293A200053657420486F70206368616EBA
:100690006E656C7320286D61782032342C20736570
:1006A0007061726174656420627920636F6D6D6141
:1006B00073292076616C69642076616C756573209E
:1006C000312D3235353A2000536574206368616EF0
:1006D0006E656C2073706163696E672028783130B5
:1006E0006B487A293A200053657420524620706F77
:1006F0007765722028302D37293A20005365742001
:100700005246206D616769632028686578292065F5
:100710002E672E20307844454144463030443A20FC
:10072000005365742062617365206672657175653A
:100730006E63792028696E20487A293A20005B5A36
:100740005D20656E74657220726563656976657299
:1007500020636F6E66696775726174696F6E20756C
:1007600074696C79005B465D20646973706C6179B3
:100770002061637475616C206672657175656E6366
:100780006965732075736564005B525D2063616CFD
:1007900063756C6174652072616E646F6D206B654A
:1007A0007920616E6420686F70206C697374005BDF
:1007B000495D207265696E697469616C697A65204A
:1007C00073657474696E677320746F20736B6574DE
:1007D00063682064656661756C7473005B585D20A6
:1007E000726576657274206368616E6765732061F7
:1007F0006E642065786974206D656E75005B535D6D
:1008000020736176652073657474696E67732074F4
:100810006F20454550524F4D20616E6420657869C8
:1008200074206D656E7500557365206E756D62651B
:100830007273205B302D395D20746F20656469749C
:1008400020706172616D657465727300202D205394
:10085000797374656D20636F6E6669677572617414
:10086000696F6E000A0A6F70656E4C52536E672096
:10087000005129204F7574707574206265666F721F
:1008800065206C696E6B20283D465329203A200074
:10089000502920536C617665206D6F646520286552
:1008A00078706572696D656E74616C293A20004FCD
:1008B000292054696D65642042494E4420617420AA
:1008C0007374617274757020203A20004E29205094
:1008D000504D206F7574707574206C696D69746506
:1008E0006420202020203A200044495341424C45B6
:1008F00044004D292050504D205253534920746FCD
:10090000206368616E6E656C202020203A20004CC8
:10091000292050504D206D696E696D756D20737979
:100920006E63202875732920203A200044495341E2
:10093000424C4544004B29204661696C73616665F1
:1009400020626561636F6E20696E74762E20283197
:100950002D32353573293A20004A29204661696CC9
:100960007361666520626561636F6E2064656C61AA
:10097000792028302D323535203D3E20313073200E
:100980002D203135306D696E293A200049292046E5
:1009900061696C7361666520626561636F6E206674
:1009A00072712E203A200048292050574D20737430
:1009B0006F702064656C6179202020202020203A0F
:1009C000200047292050504D2073746F70206465BB
:1009D0006C6179202020202020203A200046292008
:1009E0004661696C736166652064656C617920207D
:1009F00020202020203A200050574D206368616E4F
:100A00006E656C200066756E6374696F6E3A2000C7
:100A10002920706F72742000506F776572546F7761
:100A2000657200445446205548462033322D626991
:100A3000742031306368004F70656E4C52536E679E
:100A40005258206D696E6920342F36636800466CF9
:100A50007974726F6E2F4F72616E676552582055B0
:100A600048462038636800525820747970653A20EF
:100A70000044697361626C656400487A00203D3D02
:100A8000200043616C63756C617465642070616300
:100A90006B657420696E74657276616C3A200042F1
:100AA00029204D6963726F202868616C6629205087
:100AB000504D202020203A00412920496E76657251
:100AC0007465642050504D20696E20202020203A0B
:100AD000003029204D7574652062757A7A65722020
:100AE000286D6F73746C79293A0039292053657227
:100AF00069616C2062617564726174653A00736D3E
:100B0000617274506F7274004672536B7900547244
:100B1000616E73706172656E740044697361626CBA
:100B200065640038292054656C656D657472793A86
:100B300020202020202020003729204368616E6E6D
:100B4000656C20636F6E6669673A20200036292045
:100B500044617461726174652028302D32293A2015
:100B6000202000352920486F70206368616E6E6513
:100B70006C733A2020202020003429204368616EC5
:100B80006E656C2073706163696E673A2020003374
:100B90002920524620706F7765722028302D372922
:100BA0003A202020003229205246206D6167696377
:100BB0003A202020202020202020003129204261BE
:100BC0007365206672657175656E63793A202020C1
:100BD0000000000000240027002A0000000000257B
:100BE0000028002B0000000000230026002900043C
:100BF00004040404040404020202020202030303C4
:100C000003030301020408102040800102040810BD
:100C1000200102040810200000000700020100006B
:100C2000030406000000000000000000232F112430
:100C30001FBECFEFD8E0DEBFCDBF13E0A0E0B1E034
:100C4000E8E8F0E602C005900D92A839B107D9F79F
:100C500016E0A8E9B3E001C01D92AB35B107E1F79A
:100C60001CE0CEE2DCE004C02297FE010E941F30AF
:100C7000CC32D107C9F70E94682F0C9442300C94F3
:100C80000000A0E0B0E0E7E4F6E00C94EE2FEC0109
:100C9000A880B980CA80DB80A114B104C104D1044A
:100CA00041F484E2A82E89EDB82E8BE5C82E87E0AA
:100CB000D82EC601B5012DE133EF41E050E00E948E
:100CC000CB2F27EA31E440E050E00E94772F7B01F0
:100CD0008C01C601B5012DE133EF41E050E00E94E7
:100CE000CB2FCA01B9012CEE34EF4FEF5FEF0E941A
:100CF000772F6E0D7F1D801F911F97FF04C06150DD
:100D0000704080409048688379838A839B839B01ED
:100D1000AC015F77B901CA01CDB7DEB7EAE00C9448
:100D20000A300E944106089581EB92E00E9441063C
:100D300008956093B1027093B2028093B3029093CE
:100D4000B4020895A0E0B0E0E8EAF6E00C94E72FE2
:100D5000EC012B016A016115710519F0FB0191830A
:100D60008083C114D10449F0C6010297839728F00B
:100D700020E030E040E050E0DCC0A9908A2D90E017
:100D80000E943730892BC9F7FDE2AF1621F4A990F4
:100D90003324339405C08BE2A81609F4A9903324B8
:100DA000C114D10421F0E0E1CE16D10411F5F0E335
:100DB000AF1669F48881883711F0883541F4A9802D
:100DC000229682E0382A20E1C22ED12C12C0C11412
:100DD000D10479F4E0E3AE1659F199E9E92E99E9E5
:100DE000F92E99E9092F99E1192F8AE0C82ED12C03
:100DF0003AC0FAE0CF16D10491F080E1C816D104D0
:100E000029F0E8E0CE16D104F9F415C0BFEFEB2EBF
:100E1000BFEFFB2EBFEF0B2FBFE01B2F24C0A9E9B4
:100E2000EA2EA9E9FA2EA9E90A2FA9E11A2F1BC077
:100E3000F8E0CF2ED12CEFEFEE2EEFEFFE2EEFEFFE
:100E40000E2FEFE11E2F0FC09601442737FD40956E
:100E5000542F6FEF7FEF8FEF9FEF0E94A92FC901F3
:100E6000DA017C018D0120E030E040E050E060E0FC
:100E70003601882477FC8094982C70EDB72EBA0C3C
:100E8000F9E0FB1570F48A2D81548A3118F499EC3D
:100E9000B92E06C08A2D81568A3148F589EAB82EC6
:100EA000BA0C8B2D90E08C159D050CF56F3FE9F089
:100EB000E216F30604071507B8F0CA01B901A40148
:100EC00093010E94772F9B01AC018B2D90E0A0E055
:100ED000B0E0280F391F4A1F5B1F281739074A0740
:100EE0005B0710F061E001C06FEFA990C6CF41141D
:100EF000510451F0662311F0219703C031FE04C064
:100F00002297F201D183C08330FE07C050954095EF
:100F1000309521953F4F4F4F5F4F67FF0AC082E2E8
:100F200090E090935A06809359062FEF3FEF4FEFD2
:100F30005FEFB901CA01CDB7DEB7E1E10C94033030
:100F4000FC0188279927E89421912032E9F3293080
:100F500010F02E30C8F32B3241F02D3239F4689462
:100F600004C00E94F507820F911D219120532A3061
:100F7000C0F31EF4909581959F4F089548E953E082
:100F80000E94C3070895009731F4DA018D919C9176
:100F9000009709F40EC0DC01FB013D912191222351
:100FA00019F03217C9F3FACF332331F4DA011D9265
:100FB0001C928827992708951197AF93BF93FB013F
:100FC0003D912191321771F4332321F48827992719
:100FD000119702C01E921196FA01A193B0839F91BE
:100FE0008F910895222369F7EACF7AE0979F902D99
:100FF000879F802D910D1124089580919A0381304F
:1010000019F482E080939A0380919A03833019F453
:1010100084E080939A030895E3E0F0E089E0809310
:101020005700849190E08670863009F491E0892F12
:1010300008951F93182F0E940C08882379F09FB7FA
:1010400081E08093A105F894A89588E180936000E1
:1010500010936000112309F0A8959FBF1F91089578
:10106000382F20E080913305909134058227932713
:1010700040E061E270E19C01220F331F97FF04C042
:10108000C9018627972701C0C9014F5F483099F7EA
:101090009093340580933305089587E38093D003BC
:1010A00080E092ECA1E0B0E08093D1039093D20372
:1010B000A093D303B093D40387E08093DD0380E053
:1010C00091EAACEBB3E38093D5039093D603A0935E
:1010D000D703B093D80385E08093DE038DEE9EEFB7
:1010E000ADEABEED8093D9039093DA03A093DB03BE
:1010F000B093DC03AFEDB3E080E090E0863010F019
:10110000E0E004C0FC01EF57FC4FE081ED93019655
:101110008831910599F782E08093F7038AE0809304
:10112000F803089580E09EECADEEB4E380939D0358
:1011300090939E03A0939F03B093A00380E090E060
:10114000A0E0B0E58093A1039093A203A093A30332
:10115000B093A403E5EAF3E080E081938F5F8031F0
:10116000E1F708958436910520F4BC0180E090E019
:1011700025C08E3B910550F48A559040BC0180E01B
:1011800090E02AE030E040E050E016C0823D91055A
:1011900050F4845B9040BC0180E090E024E630E0B5
:1011A00040E050E009C08D5C9040BC0180E090E0E0
:1011B00028E532E040E050E00E94772F24E630E05E
:1011C00040E050E00E94772F089590E08C599F4FA7
:1011D0000E94B2080895DC019896EC91F0E0E77067
:1011E000F070E758FC4F808108958F929F92AF92E4
:1011F000BF92CF92DF92EF92FF920F931F938C01D9
:101200000E94EB08D80197962C9130E043E150E022
:10121000249FF001259FF00D349FF00D1124EB5415
:10122000FD4F80809180A280B38090E00F96AA2726
:1012300097FDA095BA2FBC01CD0120E43FE14DE719
:1012400050E00E94772FA50194010E94A92F690107
:101250007A0180ED97E0A0E0B0E0C80ED91EEA1E4A
:10126000FB1ED80198968C91887181F060E07EEE2B
:101270008AEB9BE0A50194010E94A92F28513C4FC5
:101280004F4F5F4FC20ED31EE41EF51E87EE93E054
:10129000A0E0B0E0C80ED91EEA1EFB1EC701B601D1
:1012A00028EE33E040E050E00E94A92FCA01B901C6
:1012B00028EE33E040E050E00E94772F1F910F911D
:1012C000FF90EF90DF90CF90BF90AF909F908F9066
:1012D00008958F3F910509F010F480E0089522E011
:1012E0008030920710F481E008958050934010F010
:1012F00083E0089582E00895CF92DF92FF920F93EA
:101300001F93CF93DF93F82FEB016A01182F1695E7
:10131000E0E088819981D6018C938A819B81119626
:101320008C9311978C819D8112968C9312978E814C
:101330009F8113968C931397288139814A815B8111
:101340006C817D818E819F819295990F990F907C00
:10135000832F8370982B852F8370880F880F982B8D
:10136000872F83708295807F982B14969C9385E0BD
:1013700090E0C80ED91E2896EF5F1E1750F6F0FFBA
:1013800021C0888199810E946909F82E8A819B81F8
:101390000E946909182F8C819D810E946909082F7C
:1013A0008E819F810E946909F294FF0CFF0C70EC02
:1013B000F7221295107F1F29182B000F000F012B09
:1013C000D6010C93DF91CF911F910F91FF90DF9089
:1013D000CF90089523E08032920718F420E030E0A7
:1013E00026C023E0883E920748F49C012F513340E9
:1013F00054E0369527955A95E1F719C027E0803DCE
:10140000920720F49C012C5D334011C028E08839FC
:10141000920718F02FEF33E00AC09C01285C374098
:1014200044E0369527954A95E1F72D503C4FC90188
:1014300008958C30910548F49C0174E0220F331F0D
:101440007A95E1F7285D3C4F17C023E0843F92076F
:1014500020F49C0124523C4F0FC024E080309207BE
:1014600018F020E938E008C09C012657334F64E0AB
:10147000220F331F6A95E1F7C90108959C01369543
:10148000279525753575821B930B9C0136952795FD
:10149000369527952373337383739373280F391FFE
:1014A000C901E4E096958795EA95E1F7820F931FCD
:1014B0008F709F7021E031E0AC01429FC001439FDB
:1014C000900D529F900D1124892F0895882339F093
:1014D0002D9800002B9A00002D9A000008952D9859
:1014E00000002B9800002D9A000008952D9A00000E
:1014F00083B12D98000090E0B4E096958795BA9559
:10150000E1F7817008950F931F93082F5C9A2D982F
:101510005C9810E0802F80780E94660A000F1F5FA1
:101520001830C1F72D981F910F9108958F770E9461
:10153000830A08950F931F93082F10E0802F80785F
:101540000E94660A000F1F5F1830C1F72D981F9187
:101550000F9108950F931F932D9880E000E0182FAE
:10156000110F0E94760A810F0F5F0830C1F71F919B
:101570000F9108950E94960A0E94AA0A5C9A089503
:101580001F93162F80680E94830A812F0E949A0A57
:101590005C9A1F9108951F931091D9031827E0EDCD
:1015A000F3E0E80FF11D89E767850E94C00A8DE32B
:1015B000612F0E94C00A82E4612F0E94C00A1F911D
:1015C000089586E20E94BA0A08950F931F938C0132
:1015D0008CE1F80164810E94C00A8DE1F801658107
:1015E0000E94C00A8EE1F80166810E94C00A80E272
:1015F000F80167810E94C00A81E2F80160850E94BB
:10160000C00A82E2F80161850E94C00A83E2F80103
:1016100062850E94C00A84E2F80163850E94C00AC4
:1016200085E2F80164850E94C00A8AE2F8016585B6
:101630000E94C00A8EE6F80166850E94C00A8FE605
:10164000F80167850E94C00A80E7F80160890E945E
:10165000C00A81E7F80161890E94C00A82E7F801A7
:1016600062890E94C00A1F910F910895EF92FF9224
:101670000F931F93CF93DF937B018C01603028E39E
:1016800072072CE982072CE1920728F520E836E959
:1016900048E950E00E94A92FE9016897B90180E06C
:1016A00090E020E839E647E65FEF0E94772F6E0D65
:1016B0007F1D801F911F32E0660F771F881F991FC3
:1016C0003A95D1F721E732E040E050E00E94A92F9F
:1016D000890180E421C020E03DE241E351E00E9425
:1016E000A92FE9016897B90180E090E020E033ED8F
:1016F0004EEC5EEF0E94772F6E0D7F1D801F911FB5
:10170000660F771F881F991F21E732E040E050E005
:101710000E94A92F890180E69E012F71622F680F18
:1017200085E70E94C00A86E7612F0E94C00A87E70A
:10173000602F0E94C00ACDB7DEB7E6E00C940E30F1
:101740009F92AF92BF92CF92DF920F93DF93CF938E
:1017500000D000D0CDB7DEB7982E83E00E94BA0A41
:101760008093F90384E00E94BA0A8093FA0386E02A
:1017700060E00E94C00A87E061E00E94C00A89E040
:101780006FE70E94C00A8AE065E00E94C00A8BE011
:1017900062E10E94C00A8CE065E10E94C00A8DE00F
:1017A0006DEF0E94C00A8EE060E00E94C00A99209E
:1017B00019F084E193E008C08091F70323E1829F50
:1017C000C00111248B549D4F0E94E50A80E36CE810
:1017D0000E94C00A82E36FE00E94C00A83E362E4D1
:1017E0000E94C00A84E36AE00E94C00A85E36AE2BC
:1017F0000E94C00A86E36DE20E94C00A87E364ED9E
:101800000E94C00A88E360E00E94C00A89E360E0A9
:101810000E94C00A992049F065E8A62E61ECB62E18
:1018200061ECC62E6EEDD62E08C0A090D903B09004
:10183000DA03C090DB03D090DC030AE38D2D9927F7
:10184000AA27BB2789839A83AB83BC83802F6981B6
:101850000E94C00A802F8B5F69810E94C00ADC2C25
:10186000CB2CBA2CAA240F5F0E3341F783E46FEF21
:101870000E94C00A84E46FEF0E94C00A85E46FEF03
:101880000E94C00A86E46FEF0E94C00A992019F0F6
:101890008DE666E003C08DE66091DD030E94C00A1C
:1018A00089E760E00E94C00A8AE76091DE030E9437
:1018B000C00A83E760E00E94C00A84E760E00E94FB
:1018C000C00A992029F060E071EA8CEB93E308C02C
:1018D0006091D5037091D6038091D7039091D8037E
:1018E0000E94360B0F900F900F900F90CF91DF91C9
:1018F0000F91DF90CF90BF90AF909F90089587E0B9
:1019000061E00E94C00A8EE764E20E94C00A88E09B
:1019100063E00E94C00A88E060E00E94C00A87E09D
:1019200065E00E94C00A85E062E00E94C00A83E090
:101930000E94BA0A8093F90384E00E94BA0A809355
:10194000FA030895582F40919E04842F90E0FC01E3
:10195000EF70F0709F012F5F3F4F74E09595879572
:101960007A95E1F72817390751F0E257FB4F50837A
:10197000842F8F5F8F70407F842B80939E04089507
:101980001F920F920FB60F9211241F932F933F9324
:101990004F935F936F937F938F939F93AF93BF9377
:1019A000CF93DF93EF93FF93C0918600D091870090
:1019B0002091E0043091E1048091BF04882309F074
:1019C00062C0BE01621B730B2091A1033091A20380
:1019D0004091A3035091A40325FD02C0769567951D
:1019E00089E0653C7807B8F1809147031CE1569582
:1019F0004795379527951A95D1F72115310541055A
:101A0000510521F421E030E040E050E090E0A0E01A
:101A1000B0E0281739074A075B07D0F480914703E5
:101A20008F3FB1F020E00EC0E22FF0E0EE0FFF1F7D
:101A3000DF01A054BB4F8D919C91E95DFC4F9183D8
:101A400080832F5F80914703281770F31092BE04A4
:101A50001092470318C082E06D3B780760F18091D7
:101A60004703803140F510914703CB010E94EA09FA
:101A7000E12FF0E0EE0FFF1FE054FB4F91838083D6
:101A80001F5F10934703D093E104C093E004FF91DC
:101A9000EF91DF91CF91BF91AF919F918F917F9106
:101AA0006F915F914F913F912F911F910F900FBEBA
:101AB0000F901F9018958FEF80934703E4CF83E03A
:101AC000809380008AE9809381008091A10386FD44
:101AD00005C0809181008064809381008FEF9FEF2B
:101AE000909389008093880080916F00806280933A
:101AF0006F0008956F3018F086958058089589E03A
:101B0000689F802D11240895882319F460E071E006
:101B100002C063E071E087E396E00E942B2D0895F8
:101B2000A0E0B0E0E6E9FDE00C94F02F182F0E9451
:101B3000DC299B01AC0180912D0590912E05A0918F
:101B40002F05B091300569017A01C81AD90AEA0A4D
:101B5000FB0AD701C60189589341A040B04010F05C
:101B600010922C0520932D0530932E0540932F05C0
:101B7000509330052091BF04822F81508230E8F5C8
:101B800080912C05882309F44FC1813011F482E043
:101B9000BCC1803108F035C1E82FF0E0E054FB4FC4
:101BA00010838F5F80932C05803109F0B0C1A2ECC7
:101BB000B4E0213039F41196EC911197E695E69551
:101BC0008C9109C08D919C911197E92FE695E6952E
:101BD000E69596958795E03140F4F0E090E0EE0FC1
:101BE000FF1FE95DFC4F918380831092BE04129623
:101BF00084E0A03DB807E9F68AC1233009F004C1AA
:101C000080912C05882321F41F3009F080C10CC17C
:101C1000883130F4E82FF0E0E154FB4F108374C1B9
:101C2000883109F0EEC0112309F0EBC0C0E0D0E02C
:101C30000BE010E0DE0163E0AA0FBB1F6A95E1F73D
:101C4000C09FB001C19F700DD09F700D1124FB018A
:101C5000E054FB4F80812181922F97709595879555
:101C6000FD01EE0FFF1FE95DFC4F91838083FB01B7
:101C7000EF53FB4F30813695369536952181422FB3
:101C80004295440F407E842F832B269526952695DA
:101C9000922F977095958795FD01EE0FFF1FE75DD9
:101CA000FC4F91838083FB01EE53FB4F8081829533
:101CB0008695869583704181942F990F990F292FCE
:101CC000282B429546954695437082818170880FF6
:101CD000880F382F342B35952795FD01EE0FFF1F08
:101CE000E55DFC4F31832083FB01EC53FB4F3081DA
:101CF00036952181422F479544274795842F832B82
:101D00002695922F977095958795FD01EE0FFF1FF1
:101D1000E35DFC4F91838083FB01EB53FB4F3081EC
:101D200032953F702181422F4295407F842F832B33
:101D300022952F70922F977095958795FD01EE0F44
:101D4000FF1FE15DFC4F91838083FB01EA53FB4F52
:101D50008081881F8827881F4181942F990F292F00
:101D6000282B441F4427441F82818370880F382FFB
:101D7000342B35952795FD01EE0FFF1FEF5CFC4FCF
:101D800031832083FB01E853FB4F30813695369534
:101D90002181422F4295440F440F407C842F832B96
:101DA00026952695922F977095958795AA0FBB1F1C
:101DB000FD01ED5CFC4F9183808367537B4FFB01FA
:101DC00020812295269527704181342F330F330FC0
:101DD000330F832F822B942F92959695977095951C
:101DE0008795AB5CBC4F11969C938E932196C23025
:101DF000D10509F01FCF8091D60483FD02C0109257
:101E0000BE0410922C0583C0243009F080C040919C
:101E10002C05442359F4183AB1F410923405109269
:101E2000330588EA0E94300881E06FC0413019F420
:101E30001093310504C0423031F410933205812FE4
:101E40000E9430085DC060913205262F30E0220FDD
:101E5000331FE42FF0E0C90102968E179F0734F07C
:101E6000433268F7E354FB4F1083E9CF2D5F3F4FB8
:101E70004091330550913405E217F30749F4912F4F
:101E800080E048275927509334054093330538C0E4
:101E9000812F90E04817590789F5809131058130ED
:101EA00069F5613118F080E180933205D0903205F8
:101EB00040ECE42E44E0F42E00E010E01BC0F701FB
:101EC000D081C0E0818190E08C2B9D2B33E09695F2
:101ED00087953A95E1F70E94EA09F801EE0FFF1F96
:101EE000E95DFC4F918380830F5F1F4F82E090E09C
:101EF000E80EF91E0D1518F31092BE0410922C0571
:101F000080912C05882319F08F5F80932C05CDB725
:101F1000DEB7E8E00C940C30FF920F931F93CF9341
:101F2000DF93182F092FF62E8EE30E94C00A212F6F
:101F3000302FC901EC0110E005C08FE769910E94C4
:101F4000C00A1F5F1F15C8F385E064E00E94C00A45
:101F500083E00E94BA0A8093F90384E00E94BA0ADF
:101F60008093FA030E94DC296093FB037093FC03C7
:101F70008093FD039093FE0387E069E00E94C00A0E
:101F800081E080939A03CDB7DEB7E5E00C940F3083
:101F90000E948C0F80919A038130D9F40E94DC2931
:101FA0002091FB033091FC034091FD035091FE030F
:101FB000621B730B840B950B605A764881409040EE
:101FC00040F4E8CF87E396E067E071E00E942B2DB4
:101FD000089580919A038130A9F3089587E396E0EC
:101FE0006EE70E94E32E0895A0E0B0E0EAEFFFE084
:101FF0000C94EF2F6C0187E396E06EE70E94E32ECE
:102000007601C0E0D0E000E010E0B0E2BB2E0AC0F4
:102010000830110521F49E012095F60120870894CF
:10202000E11CF11CF7016081862F8D57823040F44E
:1020300087E396E06DE70E94E32EF70160816B2550
:1020400087E396E00E94E32E0115110551F0F70198
:1020500080819E01280F311DC32FDD27C20FD31FA2
:10206000D0700F5F1F4F0930110591F6CDB7DEB765
:10207000E9E00C940B30A9E0B0E0E1E4F0E10C946D
:10208000F62F382FE62F8091A30490E0019664E2AA
:1020900070E00E94962F982F8093A30488E989838B
:1020A00080E18A83913071F0913028F0923099F07C
:1020B0009330E1F416C085E08B8381EF8C832F5F32
:1020C0002D8317C09B8381EF8C8384E6489FC001DA
:1020D00011249D830EC084E08B8381EF8C833D832C
:1020E00008C09B8381EF8C83ED8303C00E94EE0FB9
:1020F00004C0CE0101960E94F40F2996E2E00C94F0
:1021000012300F931F93CF93DF93182F092F87E37C
:1021100096E06EE70E94E32E212F302FC901EC01DB
:1021200010E000E288818D57823040F487E396E02A
:102130006DE70E94E32E88818027888387E396E0FD
:1021400069910E94E32E1F5F193061F787E396E0E3
:102150006EE70E94E32EDF91CF911F910F910895BA
:10216000A9E0B0E0E6EBF0E10C94F62F382F809177
:10217000A304882379F48EEF89833A836B83842FB9
:1021800090E0959587958C832D83198618861F82FC
:102190001E822FC040919E04842F90E09C012F70DE
:1021A000307054E0959587955A95E1F7821793071B
:1021B00021F18DEF89831A821B82DE01149620E0C3
:1021C00008C0E257FB4F80818D93405F2F5F263020
:1021D00069F0842F90E0FC0134E0F595E7953A959D
:1021E000E1F78F709070E817F90759F740939E0454
:1021F0002A83CE0101960E9481108091A30490E071
:10220000019666E070E00E94962F8093A3042996C1
:10221000E2E00C9412309F92AF92BF92CF92DF9285
:10222000EF92FF920F931F93B82EA62ED42EC22E9C
:10223000902E0E94DC297B018C0180918D042091DD
:102240009F043091A0044091A1045091A2048823DE
:10225000B1F0D801C701821B930BA40BB50B815EB3
:102260009E42A040B04020F12C2DDC1408F42D2D0E
:102270008B2D6A2D422F292D0E943B1011C0D801B1
:10228000C701821B930BA40BB50B81539547A0404C
:10229000B04070F08B2D6A2D4D2D2C2D0E94B0106A
:1022A000E0929F04F092A0040093A1041093A20472
:1022B0001F910F91FF90EF90DF90CF90BF90AF9064
:1022C0009F90089587E396E0609100040E94E32EBA
:1022D00008951F93182F87E396E0612F0E94E32E45
:1022E000809100048127809300041F9108951F931B
:1022F000192F0E946911812F0E9469111F91089561
:10230000DF92EF92FF920F931F93D82E7B011092D2
:10231000000407E316E0C80165EB0E94E32EC80144
:1023200062E60E94E32E8D2D0E946911C7010E9472
:1023300077111F910F91FF90EF90DF900895E82F94
:10234000F0E0E456FC4FE185E03158F4F894F0E019
:10235000EE0FFF1FE95DFC4F0190F081E02D7894B6
:102360000DC0E03129F0E13129F0E0E0F2E006C0F3
:1023700082E101C083E10E94302BFC01CF0108956E
:102380008CE060E00E94612A8BE061E00E94612A9B
:102390008DE061E00E94612A82E060E00E94612A93
:1023A00084E061E00E94612A0895EF92FF920F930A
:1023B0001F93009771F19C0140E050E068E478EED3
:1023C00081E090E00E94CB2FC901DA017C018D01F0
:1023D00083E161E00E94CD2A8FEFE816F104010548
:1023E000110539F030F0FFEFEF2EF12C012D112DFA
:1023F0000AC0E114F1040105110529F4E1E0EE2E13
:10240000F12C012D112DE092B3008091B00080617C
:1024100007C083E160E00E94CD2A8091B0008F7EEA
:102420008093B0001F910F91FF90EF900895A0E26C
:10243000B0E0EDE1F2E10C94EE2F8CE00E94BA0ADC
:10244000882379F587E396E063E171E00E942B2D04
:10245000439A80E00E94A00B0E947F0C439821C009
:1024600087E396E00E94AA2E482F8091BF0488231C
:1024700021F0842F0E94900D14C080912A05E82F2E
:10248000F0E031969F012F713070319780912905CE
:1024900090E02817390729F0E050FB4F4083209344
:1024A0002A0587E396E00E94702E892BC9F6809159
:1024B0009A03843009F08EC00E94DC296093AE0438
:1024C0007093AF048093B0049093B10461157105CB
:1024D0008105910561F481E090E0A0E0B0E0809397
:1024E000AE049093AF04A093B004B093B104809174
:1024F000BA049091BB0481609093BB048093BA04AA
:1025000083E080939A038FE70E94960A07EF14E016
:102510000E94AA0AF80181938F01F5E000301F079D
:10252000B9F74091E2048091F704282F30E0842F1E
:1025300090E08227932786FF40C080E4482740939D
:10254000E204C90188739070C89709F510E014C0BF
:102550001F5F8091F803E12FF0E084FF06C0E9508F
:10256000FB4F80810E94A20C07C0E950FB4F87E31C
:1025700096E060810E94E32E212F30E08091F704E5
:1025800090E0877090708217930714F716C02F732E
:102590003070232B91F48091F8048093B2048091E1
:1025A000F9048093B4048091FA048093B504809177
:1025B000FD048093BC041092BD0480912B058130F2
:1025C00019F482E080932B0580912B05833011F460
:1025D00010922B050E94DC295B016C018091B604EE
:1025E0009091B704A091B804B091B9040097A105E7
:1025F000B105C9F086017501E81AF90A0A0B1B0B2F
:10260000D801C701885B9B40A040B04060F00E94A9
:10261000E10A8093B3041092B6041092B7041092AA
:10262000B8041092B90480ED93E00E94F50820915F
:10263000AA043091AB044091AC045091AD048601E2
:102640007501E21AF30A040B150BE616F7060807E4
:10265000190708F40CC1A092AA04B092AB04C0926E
:10266000AC04D092AD04A8958091BE048830A0F04F
:102670008091A1039091A203A091A303B091A40320
:102680002CE1B695A795979587952A95D1F7009750
:10269000A105B10509F08AC18091BE048F5F8093C6
:1026A000BE04E090AE04F090AF040091B00410912D
:1026B000B104E114F1040105110511F180ED93E07D
:1026C0000E94F508AE18BF08C00AD10A6A157B053A
:1026D0008C059D0588F48091A10384FD04C080EDE4
:1026E00097E00E94D5111092AE041092AF041092A0
:1026F000B0041092B10404C080E090E00E94D511B3
:102700009091E204907C9093E20400912A0510914C
:1027100029050117B1F180912B05823091F5905870
:102720009093E20480ED93E00E94EB08893010F072
:1027300048E002C0482F415030E013C03F5FA32F54
:10274000B0E0812F90E0FC01E050FB4F2081FD01C3
:10275000EE51FB4F2083A05EBA4F2C930196182FA9
:102760001F71341710F4101749F710932905832FA0
:10277000895C9091E204892B8093E20430932005D8
:102780001AC020912B052430D1F490912005E1E26C
:10279000F5E0A3EEB4E0292F30E02E0F3F1F02C07A
:1027A00081918D93E217F307D9F7995C8091E20448
:1027B000982B9093E20483E080932B0536C08091A0
:1027C000A504823059F491609093E204439A05EA9B
:1027D00013E07E010894E11CF11C10C09093E20408
:1027E0004398222319F481E080932B0580912B05D7
:1027F000833069F784E080932B05E9CFF80181915C
:102800008F010E949F11F701819391937F01F3E063
:10281000053B1F0799F78091F8038770BE016F5F32
:102820007F4F43EE54E00E947C09429A8091A404B9
:102830000E94CB0A80ED93E00E94EB08682F82EEA5
:1028400094E00E948C0FE091A404EF5FE093A40455
:10285000E83131F0F0E0E053FC4F8785882339F40C
:102860001092A40404C0439A89E08093BE0480912E
:10287000F803887171F180919A03823051F580914B
:10288000BA049091BB04880F991F9093BB04809366
:10289000BA0483E080939A030E947F0C0E94DC2993
:1028A0006093B6047093B7048093B8049093B9040E
:1028B000611571058105910561F481E090E0A0E06A
:1028C000B0E08093B6049093B704A093B804B0939B
:1028D000B9048091F80384FF1EC08091BA049091DE
:1028E000BB048E7F0E943E0A182F8091B204609133
:1028F000BC040E947A0D082F8091B304612F0E94BE
:102900007A0D282F8091B4046091B504402F009176
:102910009B030E940B1142988091A5048130D1F055
:10292000813020F0823009F047C034C082E10E943B
:10293000002B892B09F040C081E08093A5040E9400
:10294000CE296093A6047093A7048093A804909363
:10295000A90432C082E10E94002B892B21F50E943C
:10296000CE292091A6043091A7044091A80450914B
:10297000A904621B730B840B950B695E7340804046
:102980009040D0F082E08093A50480ED97E00E9413
:10299000D51112C082E10E94002B892B69F080E0E2
:1029A00090E00E94D5111092A50406C08091BE044B
:1029B000883009F059CF57CFA096EAE00C940A303E
:1029C00083E161E00E94612A83E160E00E94CD2AF8
:1029D00082E08093B00085E08093B10083E061E005
:1029E0000E94612A83E060E00E94CD2A08951F932F
:1029F000182F0E94DC2960939F047093A004809399
:102A0000A1049093A20410938D04112329F440E8AB
:102A100055E260E070E004C040E051EE60E070E03C
:102A200087E396E00E94E92D1F910895ACE1B0E0A4
:102A3000ECE1F5E10C94EE2F0E94DC297B018C0186
:102A400081E00E94A00B54E7A52E6E010894C11CE2
:102A5000D11C43E0B42EA982C60161E00E94C80FD8
:102A6000B0929A030E947F0C6AEF70E080E090E0E1
:102A70000E94022A80919A03833009F07DC087E387
:102A800096E00E94702E892B09F076C00E94DC2906
:102A90006E197F09800B910B6058734C894C9140E3
:102AA00008F06AC0D8CF8FE70E94960A0E94AA0A4F
:102AB000843509F05CC089830E94AA0A182F00E0BF
:102AC00010938C0400938B040E94AA0A080F111D16
:102AD00010938C0400938B040E94AA0A80938A04AA
:102AE0000E94AA0A80938904813108F040C0FF2423
:102AF00007C00E94AA0A07591B4FF8018083F3946C
:102B00000F2D10E08091890490E0880F991F08171D
:102B1000190778F380E78983CE01019661E00E946E
:102B2000C80F83E080939A030E947F0C62E370E0F9
:102B300080E090E00E94022A80919A038330A9F0FD
:102B40008FE70E94960A0E94AA0A803581F4898341
:102B500005EB13E00E94AA0AF80181938F01F3E0CC
:102B6000003D1F07B9F781E003C082E001C083E0A8
:102B70006C96EAE00C940A3080919A03833009F055
:102B800092CFF3CF83E00E94BA0A8093F90384E0E6
:102B90000E94BA0A8093FA0387E061E00E94C00AAB
:102BA0006AE070E080E090E00E94022A0E947F0CC0
:102BB000000008950F931F93082F17C0439A64E6EF
:102BC00070E080E090E00E94022A439864E670E0A2
:102BD00080E090E00E94022A1F5F101778F36CE2F9
:102BE00071E080E090E00E94022A10E0F6CF482FCA
:102BF000392F25E00DC0F999FECF1FBA842F932FEE
:102C000092BD81BD60BD0FB6F894FA9AF99A0FBED5
:102C1000215059F0F999FECF842F932F92BD81BD99
:102C2000F89A80B5681739F7089582E00E94DA159E
:102C30000895A0E0B0E0EFE1F6E10C94E72F482E14
:102C4000562EEE24FF2488249924C0E0D0E0CC2422
:102C5000DD2416E4312E04C055245394CC24DD2405
:102C6000442069F480919B03839DE0011124BCE919
:102C7000EB2EB3E0FB2EA9E18A2E912C1DC021E0A2
:102C8000421671F480919B03839DE00111246B96A1
:102C9000F0EDEF2EF3E0FF2EE9E28E2E912C0CC02A
:102CA00032E0431649F47BE9E72E73E0F72E61E04A
:102CB000862E912CC8E1D1E03E016C0C7D1C109257
:102CC000340510923305E3011BC0552059F4F999DE
:102CD000FECFD2BDC1BDF89A80B5F701E00FF11F5C
:102CE000808307C0F701E00FF11FCE0160810E94D1
:102CF000F7150E0D1F1DF80180810E9430082196E6
:102D00009E012619022F10E008151905F0F2CE01D8
:102D10005520D9F4F999FECFD2BDC1BDF89A20B59E
:102D2000F999FECF2196D2BDC1BD2197F89A80B501
:102D300090E0B22EAA248A299B2920913305309154
:102D400034052817390759F487CF21966091340547
:102D50000E94F715CE01609133050E94F71580E2BD
:102D600091E0C80ED91E91EEC91692E0D90608F47A
:102D700077CF852DCDB7DEB7E1E10C94033080E04D
:102D800061E00E94191681E061E00E941916089521
:102D900080E060E00E941916882331F081E060E055
:102DA0000E941916882331F40E9492080E944D084F
:102DB0000E94BF16089582E061E00E9419160895EE
:102DC00082E060E00E94191680919B03843020F01D
:102DD00010929B030E94DB1608951F93182F0E94E8
:102DE000E01680919B03811731F0143020F410938A
:102DF0009B030E94DB161F9108951092670485E6DD
:102E0000E2E0F4E0DF011D928A95E9F708951F934F
:102E1000182F8F3711F08830E1F5E0916704EE2329
:102E200009F455C0E150E0936704F0E0EE5FFB4F1A
:102E3000108287E396E06DE00E94E32E10E00AC066
:102E4000E12FF0E0EE5FFB4F87E396E060810E94A8
:102E5000E32E1F5F80916704181790F387E396E0D5
:102E600060E20E94E32E87E396E06DE00E94E32E8D
:102E700010E00AC0E12FF0E0EE5FFB4F87E396E041
:102E800060810E94E32E1F5F80916704181790F302
:102E90001CC08B3119F40E94FD161FC08D30E9F063
:102EA0008A30D9F080916704843688F487E396E00D
:102EB000612F0E94E32E80916704E82FF0E0EE5F1F
:102EC000FB4F10838F5F8093670480E007C087E328
:102ED00096E067E00E94972BF8CF81E01F9108955C
:102EE0001F93CF93DF93CFEDD3E010E03BC087E398
:102EF00096E062E271E00E94282D87E396E0612F60
:102F00004AE050E00E94A52C87E396E06FE271E072
:102F10000E94282D699170E080E090E02091DE030E
:102F200030E040E050E00E94772F20E137E240E0BF
:102F300050E00E94772FDC01CB014091D5035091E6
:102F4000D6036091D7037091D803480F591F6A1FA9
:102F50007B1F87E396E02AE030E00E946C2C1F5F25
:102F6000183119F08881882311F6DF91CF911F91D4
:102F70000895EF92FF920F931F93882339F487E30C
:102F800096E061E77AE00E94B52B3BC090E00E949A
:102F9000B20824E630E040E050E00E94A92F122F52
:102FA000032FF42EE52E622F732F842F952F2AE006
:102FB00030E040E050E00E94A92F87E396E0BA019C
:102FC000A9012AE030E00E945D2C87E396E06EE2E2
:102FD0000E94972B612F702F8F2D9E2D2AE030E0BD
:102FE00040E050E00E94A92FAB01BC0187E396E0CE
:102FF0002AE030E00E945D2C87E396E063E70E94C0
:10300000C92B1F910F91FF90EF900895FF920F939E
:103010001F93CF93DF9387E396E067E67AE00E9401
:10302000762B8091B503813041F487E396E06EE41E
:103030007AE00E94B52BFF246DC0823029F487E32B
:1030400096E067E37AE0F5CF843029F487E396E0F1
:1030500063E27AE0EECF853071F787E396E068E1CE
:103060007AE0E7CFCF2DD0E0C930D1051CF06F2D2D
:10307000685C02C06F2D6F5C87E396E00E94972B1F
:1030800087E396E060E17AE00E94762BBE016F5FF5
:103090007F4F87E396E04AE050E00E94012D87E3EE
:1030A00096E065E07AE00E94762B8E010B541C4F6F
:1030B000D8011196EC91E032F8F487E396E068EFDE
:1030C00079E00E94762BF8018181803130F087E32E
:1030D00096E063E371E00E94282DCB54DC4F6981B8
:1030E00070E06F7070706F5F7F4F87E396E04AE02B
:1030F00050E00E94142D0DC0F0E0EF70F070EE0F64
:10310000FF1FE75BFC4F6081718187E396E00E94BF
:103110002B2DF39480918A04F81608F4A3CF87E34B
:1031200096E06DED79E00E94762B8091CD030E94B0
:10313000B91787E396E062EC79E00E94762B8091E4
:10314000CE030E94B91787E396E067EA79E00E9410
:10315000762B8091CF030E94B91787E396E06CE845
:1031600079E00E94762B4091C5035091C60360918F
:10317000C7037091C803411551056105710539F107
:1031800087E396E02AE030E00E946C2C87E396E02B
:1031900069E579E00E94762B8091C9030E94E508D9
:1031A000AB01BC0187E396E02AE030E00E946C2C82
:1031B00087E396E065E379E00E94762B87E396E06B
:1031C0006091CA034AE050E00E94B72C06C087E332
:1031D00096E06CE279E00E94B52B87E396E06FE021
:1031E00079E00E94762B6091CB037091CC0387E34A
:1031F00096E04AE050E00E94912C87E396E062EF6F
:1032000078E00E94762B6091C403603450F470E043
:103210006F5F7F4F87E396E04AE050E00E94142DF5
:1032200006C087E396E069EE78E00E94B52B87E35D
:1032300096E06CEC78E00E94762B8091C30380FDD1
:1032400003C065E371E002C069E371E087E396E0E3
:103250000E942B2D87E396E06FEA78E00E94762BA0
:103260008091C30382700E94840D87E396E060E939
:1032700078E00E94762B8091C30384700E94840DB5
:1032800087E396E061E778E00E94762B8091C303A4
:1032900088700E94840DCDB7DEB7E5E00C940F3046
:1032A0001F93CF93DF9387E396E06BEB7BE00E9465
:1032B000762B4091D5035091D6036091D70370913E
:1032C000D80387E396E02AE030E00E946C2C87E385
:1032D00096E065EA7BE00E94762B4091D9035091FD
:1032E000DA036091DB037091DC0387E396E020E171
:1032F00030E00E946C2C87E396E06FE87BE00E9450
:10330000762B87E396E06091DD034AE050E00E946F
:10331000B72C87E396E069E77BE00E94762B87E392
:1033200096E06091DE034AE050E00E94B72C87E30C
:1033300096E063E67BE00E94762BCFEDD3E010E0D1
:1033400012C0112331F087E396E06DE371E00E9433
:10335000282D87E396E069914AE050E00E94A52C71
:103360001F5F183119F08881882359F787E396E0A9
:103370000E949F2B87E396E06DE47BE00E94762B12
:1033800087E396E06091F7034AE050E00E94B72C93
:1033900087E396E068E37BE00E94762BE091F803F8
:1033A000F0E0E770F070EE0FFF1FE759FC4F60810F
:1033B000718187E396E00E942B2D87E396E063E21C
:1033C0007BE00E94762B8091F80390E088719070EA
:1033D0008830910589F0893091051CF4892B39F0EA
:1033E0001BC08031910569F04897B1F40FC087E3A5
:1033F00096E06AE17BE00EC087E396E06EE07BE05A
:1034000009C087E396E068E07BE004C087E396E0CC
:103410006EEF7AE00E94B52B87E396E06AEE7AE0E1
:103420000E94762B4091D1035091D2036091D30337
:103430007091D40387E396E02AE030E00E946C2C80
:1034400087E396E061ED7AE00E94762B8091A103FC
:1034500080710E94840D87E396E068EB7AE00E9419
:10346000762B8091A10380740E94840D87E396E0FF
:103470006FE97AE00E94762B8091A10380720E940E
:10348000840D87E396E062E87AE00E94762B80ED77
:1034900093E00E94F508AB01BC0187E396E02AE0C7
:1034A00030E00E945D2C87E396E06DE77AE00E94B1
:1034B000762B80ED93E00E94F5089B01AC0160E45F
:1034C00072E48FE090E00E94A92F87E396E0BA01B2
:1034D000A9012AE030E00E945D2C87E396E06AE7CC
:1034E0007AE00E94B52BDF91CF911F910895EF9262
:1034F000FF920F931F937C0107E316E0C8016F2D25
:1035000070E04AE050E00E94802CC8016EE20E9408
:10351000972BB70124E0769567952A95E1F76F70B0
:103520007070C8014AE050E00E94802CC8016EE231
:103530000E94972B8FE0E822FF24C801B7014AE0E0
:1035400050E00E94802C1F910F91FF90EF90089502
:103550000F931F93CF93DF93209101042F3FA9F581
:1035600087E396E061EF75E00E94762B81E793E0B8
:103570000E94771A87E396E060ED75E00E94762B53
:1035800080918B0490918C040E94771A87E396E0D7
:103590006DE975E00E94B52B87E396E06AE775E078
:1035A0000E94B52B87E396E062E675E00E94B52B9A
:1035B00087E396E06DE375E00E94B52B87E396E024
:1035C0000E949F2B0E94061869C012160CF066C05C
:1035D000332727FD309580918A0490E08217930766
:1035E0000CF45CC087E396E068E275E00E94762BFD
:1035F00060910104772767FD709587E396E04AE0C4
:1036000050E00E94142D87E396E06DEF74E00E9475
:10361000762B08E210E03AC0C12FD0E0CC0FDD1FBE
:10362000C759DB4F288130E080910104992787FD3D
:10363000909501972817390741F587E396E06FE3E6
:1036400071E00E94282D87E396E0602F4AE050E069
:103650000E94A52C87E396E063E471E00E94282D88
:10366000E981F0E0EF70F070EE0FFF1FE75BFC4FB9
:103670006081718187E396E00E94282D87E396E0C0
:1036800067E471E00E94282D0F5F1F5F809189041D
:10369000181710F287E396E00E949F2BDF91CF91DD
:1036A0001F910F910895ACE1B0E0E9E5FBE10C94C6
:1036B000F02F282F809101048F3F09F042C1822F03
:1036C00090E0FC013A97EF36F10508F033C1EC5C6D
:1036D000FF4F0C941D3087E396E069E471E0AEC0C3
:1036E00087E396E069E471E00E942B2D1CC187E31B
:1036F00096E065E571E00E942B2D85E78983DE0168
:103700001296E5EBF3E08BE101900D928150E1F729
:10371000CE0101966CE10E94C80F0E947F0C83E0ED
:1037200080939A0368EC70E080E090E00E94022AA7
:1037300080919A03843009F0FDC08FE70E94960AB9
:103740000E94AA0A8983853509F0F4C087E396E0D0
:103750006FED74E00E94B52B87E396E061EC74E0B6
:103760000E94B52B87E396E063EA74E0ACC087E380
:1037700096E06DE671E00E942B2D89E68983CE01EB
:10378000019661E00E94C80F0E947F0C83E0809345
:103790009A0368EC70E080E090E00E94022A809139
:1037A0009A03843009F0C6C08FE70E94960A0E94EF
:1037B000AA0A89838E010E5F1F4FBDE1EB2EF12C0B
:1037C000EC0EFD1E0E94AA0AD8018D938D01AE1544
:1037D000BF05C1F7A5EBB3E0FE0132968BE1019086
:1037E0000D928150E1F78981893409F0A3C087E304
:1037F00096E065E874E00E94B52B87E396E067E603
:1038000074E00E94B52B87E396E069E474E05BC046
:1038100087E396E067E871E00E942B2D8EEF80939E
:10382000010488C020522750922F905380918A041F
:10383000891738F487E396E066E971E00E942B2D42
:1038400079C0909301046FC084E18093010487E301
:1038500096E062E174E037C085E18093010487E37C
:1038600096E06BED73E02FC086E18093010487E35F
:1038700096E064EA73E027C087E18093010487E360
:1038800096E06AE573E01FC088E18093010487E356
:1038900096E069E473E017C089E18093010487E34F
:1038A00096E065E373E00FC08AE18093010487E34B
:1038B00096E060E273E007C08BE18093010487E348
:1038C00096E068EF72E00E94B52B34C087E396E083
:1038D0006EED72E00E94B52B8091C30391E01DC094
:1038E00087E396E068EC72E00E94B52B8091C303F9
:1038F00092E013C087E396E063EB72E00E94B52B81
:103900008091C30394E009C087E396E068E972E020
:103910000E94B52B8091C30398E089278093C3034D
:103920008FEF809301040E94A81A04C087E396E0F9
:103930000E94AA2E87E396E00E94702E892BB1F791
:1039400062C1822F0E940717882309F45CC180910D
:103950006704882321F48FEF809301044CC182E037
:1039600094E060E070E040E050E00E94A2069B011D
:10397000AC0160910104862F992787FD9095A92FAE
:10398000B92FFC013197EB31F10508F024C1ED5559
:10399000FF4F0C941D30E62FFF27E7FDF095809137
:1039A0008A0490E08E179F070CF415C1DA01C90153
:1039B0000197A109B1098097A105B10548F0A8E2D6
:1039C000FA2E00E010E06F010894C108D10825C06C
:1039D000EB54FC4F822F81508083E5C0612F70E053
:1039E000660F771F67597B4FFB01808190E08C1534
:1039F0009D0591F48F2D90E0A0E0B0E08217930731
:103A0000A407B50741F4F601EB54FC4FDB01119616
:103A10008C91818301E0F3941F5F809189041817D2
:103A2000E8F2BFC02F3F31054105510511F008F004
:103A3000D2C02093CD03B7C02F3F310541055105BA
:103A400011F008F0C8C02093CE03ADC02F3F310560
:103A50004105510511F008F0BEC02093CF03A3C06B
:103A6000809102048062803719F583E094E060E081
:103A700070E040E050E00E94A2069B01AC01DC0136
:103A8000CB010197A109B1090897A105B10508F07B
:103A9000B5C0CA01B90124ED30E340E050E00E9416
:103AA000772F9B01AC012A5E3C4A4A46554E24C002
:103AB000863611F583E094E060E070E040E050E08D
:103AC0000E94A2069B01AC01DC01CB010197A10978
:103AD000B1090797A105B10508F090C0CA01B90165
:103AE00028EA31E640E050E00E94772F9B01AC01CC
:103AF000245E3C434E46544E211531054105510587
:103B000061F0DA01C90180509447AB48B24381505B
:103B10009A45A246B24008F05EC02093C503309398
:103B2000C6034093C7035093C8033DC02F3F3105E0
:103B30004105510511F008F04EC02093C90333C070
:103B4000DA01C9010197A109B1098F3F9105A105CA
:103B5000B10508F040C02093CA0325C0DA01C901AD
:103B6000845C9940A040B0408D549D41A040B0403D
:103B700030F43093CC032093CB0301E001C000E08C
:103B8000211531054105510511F48FEF07C021348E
:103B900031054105510528F4822F81508093C403DB
:103BA00002C00023C1F0809168048823D1F4809181
:103BB000D9039091DA03A091DB03B091DC03019665
:103BC000A11DB11D8093D9039093DA03A093DB0369
:103BD000B093DC0306C087E396E068EA71E00E94D8
:103BE0002B2D0E94FD168FEF8093010487E396E052
:103BF0006AE00E94C92B0E94A81A05C021E030E0AB
:103C000040E050E07ECF6C96E8E00C940C3087E307
:103C100096E06CE472E00E94B52B87E396E064E3E3
:103C200072E00E94B52B87E396E00E94702E892BEC
:103C300031F087E396E00E94AA2E0E94531B0E9457
:103C40001615823019F0833069F405C087E396E0D9
:103C500066E172E004C087E396E06FEF71E00E94D6
:103C6000B52B08958FEF80930104109268040E9491
:103C7000A81A0CC087E396E00E94702E892B31F0C1
:103C800087E396E00E94AA2E0E94531B80910104B4
:103C90008E3F81F7089580910104992787FD9095C3
:103CA000A92FB92FFC013196EB30F10508F074C053
:103CB000E254FF4F0C941D3087E396E064E678E011
:103CC0000E94B52B81E793E00E94771A87E396E084
:103CD0006CE478E00E94B52B87E396E067E278E039
:103CE0000E94B52B87E396E06DEF77E00E94B52B3D
:103CF00087E396E06CED77E00E94B52B87E396E0D2
:103D00006FEA77E00E94B52B87E396E069E877E0F9
:103D10000E94B52B87E396E065E677E00E94B52B1D
:103D200087E396E06EE377E00E94B52B87E396E0A9
:103D30000E949F2B0E9450192FC087E396E061E2FA
:103D400077E028C087E396E06CEF76E023C087E356
:103D500096E067EE76E01EC087E396E068EC76E0DA
:103D600019C087E396E064E876E014C087E396E044
:103D70006FE676E00FC087E396E06AE576E00E94A2
:103D8000B52B87E396E064E176E004C087E396E034
:103D90006EEF75E00E94B52B6AE070E080E090E085
:103DA0000E94022A04C087E396E00E94AA2E87E3BD
:103DB00096E00E94702E892BB1F70895A2E2B0E040
:103DC000E4EEFEE10C94E62F8E010F5F1F4F80E1C1
:103DD000D8011D928A95E9F787E396E066EC71E0D9
:103DE0000E942B2D0E94C21520E034E74BE852E3DD
:103DF0002F8F38A349A35AA380E09EECADEEB4E325
:103E00008B8F9C8FAD8FBE8F24EF31E040E050E070
:103E10002F8B388F498F5A8F30E5C32E33ECD32E3A
:103E2000E12CF12C412C24E7522E2BE8622E22E3C8
:103E3000722E88249924540133241E8A1D8A198ADB
:103E40001A8A1B8A1C8AFFC087E396E00E94AA2E6A
:103E50008434B9F0853430F48332B9F18C3209F00E
:103E6000CCC044C0833509F0C8C02F8D38A149A10A
:103E70005AA1C901DA012C013D0188249924540179
:103E8000E2C087E396E064E40E94972B87E396E024
:103E900040E054E76BE872E32AE030E00E94CB2C6C
:103EA00087E396E06CE20E94972B87E396E040E080
:103EB0005EEC6DEE74E32AE030E00E94CB2C87E3E9
:103EC00096E06CE20E94C92BBEC019821A821B8246
:103ED0001C821D821E821F82188619861A861B86E6
:103EE0001C861D861E861F86188A3AC0339434E0CD
:103EF000331609F0A8C069817A818B819C8128EEF4
:103F000033E040E050E00E94772F6F8F78A389A3C1
:103F10009AA36D817E818F8198850E94772F6B8F08
:103F20007C8F8D8F9E8F89859A85AB85BC858F8B85
:103F3000988FA98FBA8F6D857E858F8598890E940D
:103F4000772F6B017C0190E2C9169EE4D90690E0C0
:103F5000E90690E0F90630F48CE162E30E94C00AC1
:103F6000332471C0A0E3CA16A5E7DA06A0E0EA068A
:103F7000A0E0FA0618F48CE162E2F0CFB0E4CB16D0
:103F8000BCE9DB06B0E0EB06B0E0FB0618F48CE120
:103F900066E2E4CFE0E5CE16E3ECDE06E0E0EE0616
:103FA000E0E0FE0618F48CE162E1D8CFF0E6CF162F
:103FB000FAEEDF06F0E0EF06F0E0FF0618F48CE121
:103FC00065E1CCCF20E7C21621E1D20621E0E2066E
:103FD00020E0F20618F48CE161E0C0CF30EAC316AD
:103FE00036E8D30631E0E30630E0F30618F48CE15E
:103FF00063E0B4CF8CE165E0B1CF90ED292E280EBF
:1040000049E0421500F1032D10E0000F111F000FD1
:10401000111F81E090E08C0F9D1F080F191FD80120
:104020006D917D918D919C912AE030E040E050E0CF
:104030000E94772F620D711D811D911DF801608313
:1040400071838283938387E396E00E94702E892B8D
:1040500009F0FACE81149104A104B10489F4C301DA
:10406000B2010E94360B61E070E080E090E00E94B7
:10407000022AFFEFFE8B1D8A198A1A8A1B8A1C8A64
:104080002F89388D498D5A8D82169306A406B50660
:10409000E0F40E94E10A29893A894B895C89280F5A
:1040A000311D411D511D298B3A8B4B8B5C8B3D89FA
:1040B000381708F48D8B4E89841708F48E8B08947A
:1040C000811C911CA11CB11C56C0C301B20128EE79
:1040D00033E040E050E00E94A92F87E396E0BA0168
:1040E000A9012AE030E00E945D2C87E396E06CE2B3
:1040F0000E94972B87E396E06D894AE050E00E948A
:10410000A52C87E396E06CE20E94972B69897A8957
:104110008B899C89A50194010E94A92F87E396E0D1
:10412000BA01A9012AE030E00E945D2C87E396E005
:104130006CE20E94972B87E396E06E894AE050E09C
:104140000E94A52C87E396E06CE20E94C92B4C0CE0
:104150005D1C6E1C7F1C8B8D9C8DAD8DBE8D841562
:104160009505A605B70520F44F8C58A069A07AA044
:104170008824992454012F8D38A149A15AA1285E81
:1041800033404040504009F05ECFA296E2E10C94EB
:104190000230AAE5B0E0EFECF0E20C94F22F8B01D4
:1041A0007A018B3009F426C18C3040F5853009F452
:1041B00084C0863080F4823009F459C0833020F402
:1041C000813009F050C242C0833009F461C08430AC
:1041D00009F049C265C0883009F49DC0893038F4BF
:1041E000863009F486C0873009F03DC28CC0893022
:1041F00009F499C08A3009F036C2C9C0893609F479
:1042000082C18A3680F4863609F42DC1873620F4BF
:10421000853609F028C20EC1873609F43DC18836BB
:1042200009F021C241C18C3609F4C4C18D3638F47D
:104230008A3609F473C18B3609F015C2AFC18D36C9
:1042400009F4ECC1873C09F00EC200C281E069E2CA
:1042500070E00E94801100ED13E0F80181918F0160
:104260000E946911F3E0093F1F07B9F704C282E019
:104270006BE170E00E94801105EB13E0F801819181
:104280008F010E946911F3E0003D1F07B9F7F3C1E8
:1042900083E061E070E00E9480110E941615E9C180
:1042A00084E061E070E00E94801181E00E94691169
:1042B0000E9462110E94DE1EE0C16091890470E0DC
:1042C000660F771F85E00E94801100E010E008C0B3
:1042D000F801E759FB4F80810E9469110F5F1F4F62
:1042E0008091890490E0880F991F0817190780F3BF
:1042F000C2C186E062E070E00E94801181E793E035
:104300000E947711B8C187E061E070E00E948011DF
:1043100080918A04AEC188E061E070E00E94801163
:1043200080919B03A6C186E68983CE01019661E058
:104330000E94C80F0E947F0C83E080939A0368EC70
:1043400070E080E090E00E94022A80919A0384301D
:10435000E1F48FE70E94960A0E94AA0A89838634B4
:1043600071F489E060E270E00E94801110E00E9428
:10437000AA0A0E9469111F5F1032C9F77CC189E047
:1043800061E070E00E948011C7C089E06DC18AE0E1
:1043900069E170E00E94801181E080939C0380912C
:1043A000A105882351F08091A1039091A203A091CF
:1043B000A303B091A403806809C08091A1039091E8
:1043C000A203A091A303B091A4038F778093A103CC
:1043D0009093A203A093A303B093A4030CE913E06A
:1043E000F80181918F010E946911F3E0053B1F07DD
:1043F000B9F741C18BE061E270E00E9480118091C9
:10440000BE048F3F39F08091BE048F5F8093BE045D
:10441000815002C08091BE040E94691110E0812F7A
:104420000E949F110E94190A0E9477111F5F10318C
:10443000B1F721C185E661E070E00E948011093288
:10444000110509F015C120E030E0F901E053FC4FFF
:10445000D701A20FB31F8C9180832F5F3F4F29326A
:10446000310599F759C086E661E070E00E9480113D
:104470000B31110509F0FCC020E030E0F901EB54EC
:10448000FC4FD701A20FB31F8C9180832F5F3F4F4A
:104490002B31310599F740C087E661E070E00E945A
:1044A00080110E94BF1638C088E661E070E00E946B
:1044B000801185E78A83DE011396E5EBF3E08BE15B
:1044C00001900D928150E1F7CE0102966CE10E94BD
:1044D000C80F0E947F0C83E080939A0360E273E030
:1044E00080E090E00E94022A80919A03843009F0D3
:1044F000BFC08FE70E94960A0E94AA0A8A83853568
:1045000009F0B6C009C089E661E070E00E94801140
:104510000E944D080E94920881E0ABC08AE661E0EB
:1045200070E00E94801189E68E8FCE014E9661E088
:104530000E94C80F0E947F0C83E080939A0360E280
:1045400073E080E090E00E94022A80919A03843018
:1045500009F08EC08FE70E94960A0E94AA0A8E8FE9
:104560008E01015E1F4F4AE3E42EF12CEC0EFD1E7E
:104570000E94AA0AF80181938F01EE15FF05C1F789
:10458000A5EBB3E0FE017F968BE101900D92815087
:10459000E1F78E8D893409F06BC0BECF8BE661E008
:1045A00070E00E948011F70180810E94ED160E9448
:1045B000C816B2CF8CE661E070E00E948011003234
:1045C000110571F487E68AAFDE01DB96F70180E220
:1045D00001900D928150E1F7CE01CA9661E205C0CB
:1045E00087E48AAFCE01CA9661E00E94C80F0E949C
:1045F0007F0C83E080939A036CE474E080E090E0A9
:104600000E94022A80919A03843091F58FE70E94DC
:10461000960A0E94AA0A873459F57ECF8DE661E09A
:1046200070E00E9480110931110511F520E030E0A1
:10463000F901E456FC4FD701A20FB31F8C91808380
:104640002F5F3F4F2931310599F766CF87EC61E045
:1046500070E00E94801181E00E9469110E94621145
:104660001092FF030AC08AEC61E070E00E948011A2
:1046700080E00E9469110E946211C65ADF4FE6E095
:104680000C940E30A0E0B0E0E8E4F3E20C94EE2FDE
:1046900084E0A82E06E0B02E15E0C12E05E315E05B
:1046A000B4E6DB2EA2E0EA2EF3E0FF2EA1C087E302
:1046B00096E00E94AA2E982F8093A00580919F05D6
:1046C000833021F1843028F4813099F08230B8F4BD
:1046D00009C0853009F448C0853020F1863009F0E2
:1046E00087C05FC0953B09F083C081E080939F0540
:1046F0007FC0923609F07AC0E0929F0579C090930E
:104700009E0590939D05F0929F0572C090939B0526
:1047100010929C0580919D05892780939D05A0920C
:104720009F0566C0D92FC0E020919B0530919C0564
:104730002C2B3D2B30939C0520939B0580919D0550
:10474000892780939D05C0929F052536310508F481
:104750004FC08CEC61E070E00E94801181E00E940B
:1047600069110E94621142C02091990530919A0509
:10477000F901EB5CFA4F908380919D058927809326
:104780009D052F5F3F4F30939A05209399058091A7
:104790009B0590919C052817390750F1B0929F0511
:1047A00027C080919D05891759F4609199057091F2
:1047B0009A0580919E0545E355E00E94C9200DC0F1
:1047C0008BEC62E070E00E94801180919E050E9457
:1047D0006911809100040E946911F8018D2D1192D8
:1047E0008A95E9F710929A051092990510929F0503
:1047F00087E396E00E94702E892B09F058CFCDB741
:10480000DEB7EAE00C940A3081E08093FF0308C031
:1048100087E396E00E94702E892B11F00E944223BC
:104820008091FF038823A1F70895A0E0B0E0EBE1B9
:10483000F4E20C94F12F0E94DC29611571058105C9
:104840009105C9F30E9499061092D9031092DA03D8
:104850001092DB031092DC03DD24E090D903F0908A
:10486000DA030091DB031091DC03102F0F2DFE2CD7
:10487000EE240E9494062FEF30E040E050E00E94CA
:10488000CB2FE60EF71E081F191FE092D903F092F6
:10489000DA030093DB031093DC03D39444E0D416D3
:1048A000E1F6CFEDD3E000E010E090E1E92E97E2F1
:1048B000F92E4EC00F5F19F40E944D084DC00E94A2
:1048C000940622E330E040E050E00E94CB2F6F5F7F
:1048D000EFEDF3E090E004C08191861759F39F5FFC
:1048E0009117D0F38091DE0390E08E9D90018F9D13
:1048F000300D9E9D300D1124862F90E0AC01249F39
:10490000C001259F900D349F900D1124AA2797FD7B
:10491000A095BA2F2091D5033091D6034091D703AB
:104920005091D803820F931FA41FB51F20919D03A0
:1049300030919E0340919F035091A003281739079F
:104940004A075B0708F4B6CF69931F5F183121F05F
:104950008881882309F0AECFCDB7DEB7E7E00C94AD
:104960000D301F93109101041F3F09F0F1C08934ED
:1049700009F467C08A3428F5883309F479C089338B
:1049800068F4803309F486C0813308F06FC08B313E
:1049900009F44DC0813209F0D5C03DC0813409F41D
:1049A0009AC0823438F4893309F472C0803409F033
:1049B000C9C031C0823409F4A1C0863409F0C2C034
:1049C00052C0823609F49AC0833690F4883579F162
:1049D000893538F4823509F43FC0833509F0B2C017
:1049E0001FC08A3509F4A9C0813609F0ABC073C075
:1049F000823791F1833730F48636A9F1893609F090
:104A0000A1C01FC0883799F08A3709F496C0833750
:104A100009F098C005C087E396E069E471E019C029
:104A20000E94BF1687E396E063ED71E006C00E9426
:104A3000C81687E396E06DEE71E00E942B2D8EEF95
:104A40007FC00E944D080E94920887E396E06CE0C8
:104A500072E00E942B2D76C00E94152487E396E019
:104A600065E272E0F6CF0E9470176CC0805368C098
:104A700087E396E06CEE71E00E94B52B9091F8030D
:104A8000892F885F8871977E892B8093F80320C0D7
:104A900089E056C087E396E069ED71E00E94B52B8E
:104AA0008091A1039091A203A091A303B091A403CC
:104AB00020E130E040E050E082279327A427B5278B
:104AC0008093A1039093A203A093A303B093A403A4
:104AD0001093010437C087E396E063EC71E00E9415
:104AE000B52B8091A1039091A203A091A303B09153
:104AF000A40320E430E040E050E012C087E396E0F9
:104B000062EB71E00E94B52B8091A1039091A2030A
:104B1000A091A303B091A40320E230E040E050E074
:104B200082279327A427B5278093A1039093A203FC
:104B3000A093A303B093A40302C00E94071E8FEFAB
:104B400080930104809101048E3F09F4DDC0D4C03C
:104B50000E940717882309F4D7C08091670488232F
:104B600021F48FEF80930104C7C082E094E060E0FD
:104B700070E040E050E00E94A2069B01AC018091F1
:104B80000104992787FD9095A92FB92FFC01319732
:104B9000E930F10508F08CC0E753FF4F0C941D304D
:104BA000DA01C90181509447AB48B2438F5F994500
:104BB000A246B24008F07CC02093D5033093D603C0
:104BC0004093D7035093D8039AC02093D9033093CE
:104BD000DA034093DB035093DC0381E080936804A5
:104BE0008EC0283031054105510508F061C0209381
:104BF000DD0385C0DA01C9010197A109B1090A974E
:104C0000A105B10508F054C02093DE0378C082E00E
:104C100094E06DE371E00E94BE0710E00EC0183111
:104C200030F4E12FF0E0E053FC4F87871F5F80E016
:104C300090E06DE371E00E94BE07009759F00E947A
:104C4000A007009761F706C0E12FF0E0E053FC4FAA
:104C500017861F5F1831C0F352C02530310541055A
:104C6000510530F52093F7034AC0DA01C9010197D5
:104C7000A109B1090697A105B105D0F48091F80307
:104C8000887F822B8093F8033AC0DA01C90101972B
:104C9000A109B1098050924CA140B04048F4209342
:104CA000D1033093D2034093D3035093D40327C04E
:104CB00087E396E068EA71E00E942B2D13C0809193
:104CC000D9039091DA03A091DB03B091DC03019644
:104CD000A11DB11D8093D9039093DA03A093DB0348
:104CE000B093DC030E94FD168FEF8093010487E3ED
:104CF00096E06AE00E94C92B0E944B1E05C080917D
:104D000068048823E1F2EECF1F9108958FEF80931E
:104D10000104109268040E944B1E0CC087E396E0C9
:104D20000E94702E892B31F087E396E00E94AA2E14
:104D30000E94B124809101048E3F81F76AE070E007
:104D400080E090E00E94022A04C087E396E00E947F
:104D5000AA2E87E396E00E94702E892BB1F7089562
:104D6000AAE2B0E0E6EBF6E20C94EB2F0E94CE292B
:104D70007B018C0181E00E94A00B04C087E396E0D8
:104D80000E94AA2E87E396E00E94702E892BB1F72D
:104D90004398DD24D39452E6752E42E0842E912C64
:104DA0008C0E9D1E5E010894A11CB11C33E0C32E25
:104DB0000E94CE2920E030E06E197F09800B910B14
:104DC000693C71058105910510F021E030E08D2DE1
:104DD00090E028233923232B99F10E94CE297B01CF
:104DE0008C01429A80ED97E00E94D5117982D4011E
:104DF000E0EDF3E089E201900D928150E1F7C50109
:104E00006AE20E94C80F429880E090E00E94D511AB
:104E1000C0929A030E947F0C62E370E080E090E011
:104E20000E94022A80919A03843051F4C0929A031E
:104E30008FE70E94960A0E94AA0A823409F4DD24B0
:104E400082E10E94002B892B49F5DD24D39426C0F2
:104E5000439A429A87E396E00E94AA2E8D309105EC
:104E600069F08E3091051CF40A97B1F407C08332C3
:104E7000910569F08234910579F40CC087E396E0DE
:104E800064EA71E00E94B52B0E94862605C00E944C
:104E9000DE1E02C00E9404244398429887E396E0F5
:104EA0000E94702E892B09F483CFD2CF8F929F92CC
:104EB000AF92BF92CF92DF92EF92FF920F931F9328
:104EC00082E10E94002B892B09F083C068EC70E01E
:104ED00080E090E00E94022A80E090E00E94D511DC
:104EE0000E94CE295B016C0160ECE62E62E1F62E99
:104EF000012D112DEA0CFB1C0C1D1D1D06C082E1AD
:104F00000E94002B892B09F062C00E94CE296E15E9
:104F10007F058007910798F382E10E94002B892B7F
:104F200009F055C080ED97E00E94D5110E94CE296E
:104F30007B018C0199249394882488E496E2A0E074
:104F4000B0E0A80EB91ECA1EDB1E29C0AE14BF04F5
:104F5000C006D10638F480ED97E00E94D511882470
:104F600083941DC00E94CE296E197F09800B910B7E
:104F7000693C71058105910590F00E94CE297B0165
:104F80008C0180E0992009F481E0982E882319F49F
:104F900080E090E002C080ED97E00E94D51182E1B0
:104FA0000E94002B892B91F280E090E00E94D511A5
:104FB000882049F080919B038F5F83700E94ED16DB
:104FC0000E94C81606C00E9415240E94BF160E94A7
:104FD000B0261F910F91FF90EF90DF90CF90BF9080
:104FE000AF909F908F90089580E06DEF77E042E062
:104FF00050E00E9409290895EF92FF920F931F93AA
:1050000080E00E9419080E94C01181E161E00E94C5
:10501000612A80E161E00E94612A82E160E00E94F1
:10502000612A88E060E00E94612A88E061E00E94D5
:10503000CD2A0E94E01487E396E040E052EC61E064
:1050400070E00E94E92D0E94E0160E94C8160E949E
:105050005F0D8FEF8093BE040E94F42778940E9426
:10506000CE297B018C018091BE048F3F09F0C7C01F
:105070000E94CE296E197F09800B910B605D7740ED
:105080008040904008F0BBC0EECF87E396E00E94DE
:10509000AA2E87E396E00E94702E892BB1F787E352
:1050A00096E062E472E00E94282D81E793E00E947E
:1050B000771A87E396E069E572E00E94282D87E37E
:1050C00096E068E070E04AE050E00E94142D62E350
:1050D00070E080E090E00E94022A87E396E00E9460
:1050E000702E04970CF187E396E00E94AA2E82347A
:1050F0009105D1F487E396E00E94AA2E8E349105A3
:1051000099F487E396E00E94AA2E8434910561F415
:1051100087E396E00E94AA2E819731F480E090E028
:105120000E94D5110E94B0264091D1035091D20324
:105130006091D3037091D403DB01CA010197A109E7
:10514000B1090497A105B10568F44093BF04433049
:1051500029F040E052EC61E070E004C040EA56E81B
:1051600061E070E087E396E00E94E92D0E945627F7
:10517000439880E090E00E94D5110E945F0D80E08E
:105180000E94A00B8091A4040E94CB0A0E947F0C75
:105190001092290510922A0510922B0510E015C0D7
:1051A00062E370E080E090E00E94022A80ED97E0E8
:1051B0000E94D51162E370E080E090E00E94022A34
:1051C00080E090E00E94D5111F5F80919B038117C2
:1051D00038F78091F80390E084FF09C020E08871DF
:1051E0009070489709F421E0822F0E94F7148FE015
:1051F0000E9419081F910F91FF90EF90089580ED84
:1052000097E00E94D51182E161E00E94CD2A439A85
:1052100040CF823000F5E82FF0E0EE0FFF1FEE5593
:10522000FA4F71836083882319F08130A1F408C09C
:10523000809169008C7F842B80936900E89A08959F
:1052400080916900440F551F440F551F837F842BA5
:1052500080936900E99A08951F920F920FB60F92FA
:1052600011242F933F934F935F936F937F938F936B
:105270009F93AF93BF93EF93FF938091A20590917B
:10528000A305892B29F0E091A205F091A3050995CA
:10529000FF91EF91BF91AF919F918F917F916F910E
:1052A0005F914F913F912F910F900FBE0F901F90E4
:1052B00018951F920F920FB60F9211242F933F93C0
:1052C0004F935F936F937F938F939F93AF93BF930E
:1052D000EF93FF938091A4059091A505892B29F068
:1052E000E091A405F091A5050995FF91EF91BF917B
:1052F000AF919F918F917F916F915F914F913F916E
:105300002F910F900FBE0F901F9018951F920F9224
:105310000FB60F9211242F933F938F939F93AF93C8
:10532000BF938091AA059091AB05A091AC05B09177
:10533000AD053091AE050196A11DB11D232F2D5F46
:105340002D3720F02D570196A11DB11D2093AE05DC
:105350008093AA059093AB05A093AC05B093AD05DF
:105360008091A6059091A705A091A805B091A905E7
:105370000196A11DB11D8093A6059093A705A0934A
:10538000A805B093A905BF91AF919F918F913F91CF
:105390002F910F900FBE0F901F9018958FB7F89414
:1053A0002091AA053091AB054091AC055091AD0517
:1053B0008FBFB901CA0108959FB7F8942091A6053F
:1053C0003091A7054091A8055091A90586B5A89BE5
:1053D00006C08F3F21F02F5F3F4F4F4F5F4F9FBF62
:1053E000542F432F322F2227280F311D411D511DCD
:1053F00082E0220F331F441F551F8A95D1F7B90150
:10540000CA010895EF92FF920F931F93CF93DF93FA
:105410007B018C010E94DC29EB010EC00E94DC297B
:105420006C1B7D0B685E7340C8F30894E108F108BB
:1054300001091109C851DC4FE114F10401051105FE
:1054400069F7CDB7DEB7E6E00C940E30789484B5FA
:10545000826084BD84B5816084BD85B5826085BD70
:1054600085B5816085BDEEE6F0E080818160808356
:10547000E1E8F0E010828081826080838081816039
:105480008083E0E8F0E0808181608083E1EBF0E000
:10549000808184608083E0EBF0E0808181608083A4
:1054A000EAE7F0E08081846080838081826080838D
:1054B0008081816080838081806880831092C100B8
:1054C0000895CF93DF93482F50E0CA018D5F934F2B
:1054D000FC0134914151544FFA018491882369F1C0
:1054E00090E0880F991FFC01EF52F44FA591B49101
:1054F000FC01E552F44FC591D491662351F42FB7C6
:10550000F8948C91932F909589238C93888189238B
:105510000BC0623061F42FB7F8948C91932F909563
:1055200089238C938881832B88832FBF06C09FB7E4
:10553000F8948C91832B8C939FBFDF91CF9108952A
:10554000833071F0843028F48130A1F0823021F56D
:1055500014C08630B1F08730D1F08430E9F404C053
:10556000809180008F7703C0809180008F7D809331
:105570008000089584B58F7702C084B58F7D84BD87
:1055800008958091B0008F778093B0000895809146
:10559000B0008F7D8093B0000895FF920F931F930A
:1055A000F62E482F50E0CA01895E934FFC012491EA
:1055B000CA018D5F934FFC0114914151544FFA0180
:1055C00004910023C9F0222319F0822F0E94A02AFF
:1055D000E02FF0E0EE0FFF1FE552F44FA591B491DC
:1055E0009FB7F894FF2021F48C911095812302C07D
:1055F0008C91812B8C939FBF1F910F91FF900895E9
:105600000F931F93482F50E0CA01895E934FFC010E
:105610002491CA018D5F934FFC0104914151544F75
:10562000FA011491112319F420E030E015C022236F
:1056300019F0822F0E94A02A812F90E0880F991FD5
:105640008B51944FFC01A591B4918C9120E030E0F6
:10565000802311F021E030E0C9011F910F910895DE
:10566000982F8E3008F09E50977080914803829555
:10567000880F880F807C892B80937C0080917A0032
:10568000806480937A0080917A0086FDFCCF20911F
:10569000780040917900942F80E030E0282B392B5E
:1056A000C9010895A0E0B0E0E8E5FBE20C94F02F1A
:1056B0007C016B018A01C0E0D0E00FC0D6016D9182
:1056C0006D01D701ED91FC910190F081E02DC701B2
:1056D0000995C80FD91F015010400115110571F728
:1056E000CE01CDB7DEB7E8E00C940C30EF92FF921C
:1056F0000F931F93CF93DF937C018B01C0E0D0E029
:10570000F8010F5F1F4F6491662359F0D701ED91A7
:10571000FC910190F081E02DC7010995C80FD91FB8
:10572000EFCFCE01CDB7DEB7E6E00C940E30DC0152
:10573000ED91FC910190F081E02D09950895EF9293
:10574000FF920F931F938C016DE00E94972B7C01B9
:10575000C8016AE00E94972B9C012E0D3F1DC901D4
:105760001F910F91FF90EF900895EF92FF920F938A
:105770001F937C010E94762B8C01C7010E949F2BF6
:105780009C01200F311FC9011F910F91FF90EF90D5
:105790000895EF92FF920F931F937C010E94972B25
:1057A0008C01C7010E949F2B9C01200F311FC90152
:1057B0001F910F91FF90EF900895CF93DF93EC012D
:1057C0006115710519F420E030E00FC0DB010D9088
:1057D0000020E9F71197A61BB70BE881F981028039
:1057E000F381E02DAD0109959C01C901DF91CF91B5
:1057F00008954F925F927F928F929F92AF92BF9245
:10580000CF92DF92EF92FF920F931F93DF93CF938C
:10581000CDB7DEB7A1970FB6F894DEBF0FBECDBFF0
:105820002C01742ECB01223008F42AE019A231E2B7
:10583000C32ED12CCC0EDD1E822E9924AA24BB248B
:10584000672D752FA50194010E94A92F79018A0166
:10585000C801B701A50194010E94772F472D461B6F
:105860000894C108D1084A3010F4405D01C0495C79
:10587000F6014083E114F1040105110521F07E2CAD
:105880005F2DC801DDCFC201B6010E94DD2BA196BC
:105890000FB6F894DEBF0FBECDBFCF91DF911F9141
:1058A0000F91FF90EF90DF90CF90BF90AF909F90BF
:1058B0008F907F905F904F900895DC012115310506
:1058C00041F4ED91FC910190F081E02D642F099558
:1058D00008950E94F92B0895EF92FF920F931F9362
:1058E0007C010E945D2C8C01C7010E949F2B9C01B2
:1058F000200F311FC9011F910F91FF90EF90089564
:10590000EF92FF920F931F939A017B0100E010E04A
:10591000B801A7010E945D2C1F910F91FF90EF909D
:105920000895EF92FF920F931F937C010E94802CA9
:105930008C01C7010E949F2B9C01200F311FC901C0
:105940001F910F91FF90EF900895EF92FF920F93A8
:105950001F939A01E62EFF2400E010E0B801A70192
:105960000E945D2C1F910F91FF90EF900895EF9290
:10597000FF920F931F937C010E94A52C8C01C701FD
:105980000E949F2B9C01200F311FC9011F910F9175
:10599000FF90EF900895A0E0B0E0E1EDFCE20C9400
:1059A000F02FEC016A017B012115310541F4E881FA
:1059B000F9810190F081E02D642F09951BC02A30F8
:1059C0003105B1F477FF13C06DE20E94972B8C0173
:1059D00044275527BA014C195D096E097F09CE018C
:1059E0002AE00E94F92B9C01200F311F04C02AE0FD
:1059F0000E94F92B9C01C901CDB7DEB7E8E00C94F9
:105A00000C30EF92FF920F931F937B019A010027B6
:105A1000F7FC0095102FB801A7010E94CB2C1F9115
:105A20000F91FF90EF900895EF92FF920F931F93C5
:105A30007C010E94012D8C01C7010E949F2B9C01BB
:105A4000200F311FC9011F910F91FF90EF90089512
:105A50000E94DD2B0895EF92FF920F931F937C011C
:105A60000E94282D8C01C7010E949F2B9C01200FB2
:105A7000311FC9011F910F91FF90EF900895089574
:105A80001F920F920FB60F9211242F933F934F93B3
:105A90008F939F93EF93FF938091C00082FD1DC071
:105AA0004091C6002091EF053091F0052F5F3F4FE8
:105AB0002F7330708091F1059091F2052817390706
:105AC00071F0E091EF05F091F005E155FA4F408358
:105AD0003093F0052093EF0502C08091C600FF913E
:105AE000EF919F918F914F913F912F910F900FBE0A
:105AF0000F901F9018951F920F920FB60F921124BE
:105B00002F933F938F939F93EF93FF9320913306AF
:105B10003091340680913506909136062817390762
:105B200031F48091C1008F7D8093C10014C0E09159
:105B30003506F0913606ED50FA4F208180913506FA
:105B40009091360601968F739070909336068093ED
:105B500035062093C600FF91EF919F918F913F9161
:105B60002F910F900FBE0F901F901895A0E0B0E0FE
:105B7000ECEBFDE20C94EC2FFC011382128288EE18
:105B800093E0A0E0B0E084839583A683B7838BE89D
:105B900093E0918380837587648757874687318B2D
:105BA000208B138B028BF58AE48AD78AC68AB18E42
:105BB000A08E938E828E8F85848F8889858F898928
:105BC000868F8A89878F8B8980A32096ECE00C943E
:105BD0000830AF92BF92DF92EF92FF920F931F9324
:105BE000CF93DF93EC017A018B01DD24403081EE0D
:105BF000580780E0680780E0780711F0DD24D3942F
:105C000091E0A92EB12CEC89FD89DD2069F0C50158
:105C100008A002C0880F991F0A94E2F7808360E011
:105C200079E08DE390E005C0108260E874E88EE1D1
:105C300090E0A80197010E94A92F215030404040D8
:105C40005040569547953795279580E12030380785
:105C500020F0DD2011F0DD24D6CFE889F9893083EA
:105C6000EA89FB89208319A2EE89FF89408121E01E
:105C700030E0C9010C8C02C0880F991F0A94E2F72A
:105C8000482B4083EE89FF894081C9010D8C02C0F9
:105C9000880F991F0A94E2F7482B4083EE89FF8909
:105CA0004081C9010E8C02C0880F991F0A94E2F747
:105CB000482B4083EE89FF8980810F8C02C0220F20
:105CC000331F0A94E2F7209528232083DF91CF9198
:105CD0001F910F91FF90EF90DF90BF90AF900895CC
:105CE000DC011C96ED91FC911D97E05CFF4F21912A
:105CF000319180819181281B390B2F733070C9013C
:105D0000089587E396E00E94702E892B11F00E947F
:105D10003F2D0895DC011C96ED91FC911D97E05CF0
:105D2000FF4F20813181E054F040DF01AE5BBF4F77
:105D30008D919C9111972817390719F42FEF3FEF98
:105D400007C08D919C91E80FF91F8081282F30E0CA
:105D5000C9010895DC011C96ED91FC911D97E05C52
:105D6000FF4F20813181E054F040DF01AE5BBF4F37
:105D70008D919C9111972817390719F42FEF3FEF58
:105D800010C08D919C911197E80FF91F20818D9182
:105D90009C91119701968F73907011969C938E939E
:105DA00030E0C9010895DC0191968C919197882388
:105DB00039F05496ED91FC915597808186FFF9CF8B
:105DC00091961C920895CF93DF93EC01EE85FF85A9
:105DD000E05CFF4F20813181E054F0402F5F3F4F66
:105DE0002F733070DF01AE5BBF4F8D919C91119787
:105DF00028173907D1F3E05CFF4F80819181E0548F
:105E0000F040E80FF91F6083EE85FF85E05CFF4FEF
:105E100031832083EE89FF89208181E090E00F8C1F
:105E200002C0880F991F0A94E2F7282B208381E093
:105E300089A3EC89FD8980818064808381E090E082
:105E4000DF91CF9108958F929F92AF92BF92CF92A0
:105E5000DF92EF92FF920F931F9300D000D00F922A
:105E6000EDB7FEB7319684E0ADB7BEB711968C930F
:105E700083E0818387E0828385E0838381E084837C
:105E800087E396E06FEA75E043EF55E025EC30E0FC
:105E900004EC10E0B0ECEB2EF12CA1ECCA2ED12CCE
:105EA000F2ECAF2EB12CE6EC8E2E912C0E94B62D8A
:105EB0000F900F900F900F900F901F910F91FF90E8
:105EC000EF90DF90CF90BF90AF909F908F9008950C
:105ED000CF93DF930E94262A0E94FC27C1E8DEE2CE
:105EE0000E9417122097E1F30E94812EF9CF629F42
:105EF000D001739FF001829FE00DF11D649FE00DC2
:105F0000F11D929FF00D839FF00D749FF00D659F22
:105F1000F00D9927729FB00DE11DF91F639FB00D21
:105F2000E11DF91FBD01CF011124089597FB092E32
:105F300007260AD077FD04D086D006D000201AF4B8
:105F4000709561957F4F0895F6F7909581959F4FD5
:105F50000895A1E21A2EAA1BBB1BFD010DC0AA1FAA
:105F6000BB1FEE1FFF1FA217B307E407F50720F0C2
:105F7000A21BB30BE40BF50B661F771F881F991F3D
:105F80001A9469F760957095809590959B01AC0186
:105F9000BD01CF01089597FB092E05260ED057FDB0
:105FA00004D0D7DF0AD0001C38F4509540953095C6
:105FB00021953F4F4F4F5F4F0895F6F7909580958D
:105FC000709561957F4F8F4F9F4F08952F923F920D
:105FD0004F925F926F927F928F929F92AF92BF92F9
:105FE000CF92DF92EF92FF920F931F93CF93DF93A5
:105FF000CDB7DEB7CA1BDB0B0FB6F894DEBF0FBE02
:10600000CDBF09942A88398848885F846E847D844E
:106010008C849B84AA84B984C884DF80EE80FD8050
:106020000C811B81AA81B981CE0FD11D0FB6F894C6
:10603000DEBF0FBECDBFED010895EE0FFF1F05902F
:10604000F491E02D0994AA1BBB1B51E107C0AA1FC4
:10605000BB1FA617B70710F0A61BB70B881F991F09
:106060005A95A9F780959095BC01CD01089591119D
:1060700006C0803219F089508550D0F708959927CD
:0860800088270895F894FFCF72
:106088004E6F005965730054582074696D656F75BB
:106098007421006D6F64756C65206C6F636B65644B
:1060A8003F00486F70206368616E6E656C20002049
:1060B80040200053004E2F4100386368002C002C0C
:1060C800205B005D20280029004E4F5420454E419A
:1060D800424C45440053656E64696E67207365746D
:1060E80074696E677320746F2052580A0052657382
:1060F800657474696E672073657474696E6773205C
:106108006F6E2052580A0041626F72746564206590
:10611800646974730A00696E76616C6964207365DA
:106128006C656374696F6E000D0A496E76616C69FF
:106138006420696E707574202D20646973636172C0
:106148006465642107007363616E6E6572206D6F0C
:1061580064650053657474696E677320736176654E
:106168006420746F20454550524F4D0A00526576A1
:1061780065727465642073657474696E67732066EC
:10618800726F6D20454550524F4D0A004C6F616447
:10619800656420666163746F7279206465666175F1
:1061A8006C74730A004B657920616E6420636861C2
:1061B8006E6E656C732072616E646F6D697A65646A
:1061C8000A004F70656E4C52536E67205458207306
:1061D80074617274696E672000206F6E20485720C2
:1061E8000050504D0052535349005344410053430B
:1061F8004C00525844005458440041494E004C4207
:106208004545500053504B54524D0053425553008E
:1062180053554D44004C4C494E440000342B340037
:106228003800382B340031320031322B340031360B
:106238000001000000C01200001A400AA1204EA56B
:10624800001B1E27522C23308025000005400AA180
:10625800204EA50020244EA52C2330004B0000061C
:10626800400AD0009D49007B289D492C233000E13D
:10627800000005400A4501D7DC03B81E0EBF002305
:106288002E48E801008A400A6001555502AD1E20DB
:10629800000023C88025000005400AA1204EA50063
:1062A80020244EA52C233000020002000200020028
:1062B80002000200020002000200020002000200C6
:1062C80002000200020002FF01610265026A026E1A
:1062D80002720276027A027E0284028B0290029592
:1062E800029B029B029B029B0235019C02A002A218
:1062F80002A602A902AE02350100070B0C10111507
:1063080000160A1322312900000000E32E522B70D8
:086318002EAA2E8A2ED32E00BE
:107E00000F92CDB7DEB7112484B714BE81FFF1D035
:107E100082E08093C00088E18093C10086E0809377
:107E2000C20080E18093C4008EE0CDD088249924E4
:107E3000CC24C394F5E0DF2EE1E1EE2E73E0F72EC3
:107E4000B6D0082F813479F4B2D08983C2D0898129
:107E5000823811F481E005C0813811F485E001C059
:107E600083E09ED09AC0823411F484E103C085344B
:107E700019F485E0B6D091C0853561F498D0082F0B
:107E800010E095D090E0982E8824802A912A880CC2
:107E9000991C82C0863521F484E0A3D080E0E1CF34
:107EA000843609F04CC083D082D0A82E80D0B82E62
:107EB00000E011E07CD0F80181938F01AE16D1F77C
:107EC00088D0FB2DF53489F4E0E0F1E00BC0F9999E
:107ED000FECF92BC81BC0894811C911C819180BD15
:107EE000FA9AF99AEA1598F358C08B2D863409F05E
:107EF00054C0F401F7BEE89507B600FCFDCFF401CD
:107F0000A0E0B1E02C9130E011968C91119790E0B7
:107F1000982F8827822B932B12960C01C7BEE895C9
:107F20001124329681E0A038B80761F7F401D7BE7A
:107F3000E89507B600FCFDCFE7BEE8952EC0843774
:107F4000F1F435D034D0182F32D0B82E42D0FB2DDA
:107F5000F63421F4F40105914F010CC0FB2DF534EA
:107F600049F4F999FECF92BC81BC0894811C911C04
:107F7000F89A00B5802F14D0115049F70EC08537FC
:107F800039F427D08EE10CD085E90AD08FE069CF93
:107F9000813511F488E017D01CD080E101D050CF9A
:107FA0009091C00095FFFCCF8093C600089580910A
:107FB000C00087FFFCCF8091C00084FD01C0A89560
:107FC0008091C6000895E0E6F0E098E19083808318
:107FD0000895EDDF803219F088E0F5DFFFCF84E10E
:107FE000DFCF1F93182FE3DF1150E9F7F2DF1F9166
:0E7FF0000895282E80E0E7DFEE27FF27099492
:027FFE0001057B
:0400000300007E007B
:00000001FF
